:1000000010C01DC01CC0E3C11AC019C018C017C061
:1000100016C015C014C0DCC112C011C010C00FC082
:100020000EC011241FBECFEDCDBF10E0A0E6B0E0A2
:1000300001C01D92A436B107E1F74ED01EC2E0CF39
:10004000A89584B7877F84BF88E10FB6F89481BDF7
:1000500011BC0FBE8AB388638ABBB99AC09AD29A80
:10006000D79ADE9A83B7846083BF87B187B983E26A
:1000700086B91C9A089A8BB780628BBF80B5816065
:1000800080BD0895882321F4DD9A8BB3877E0EC04E
:10009000813021F4DC9A8BB3877D08C0823021F453
:1000A000DB9A8BB38F7C02C08BB3877C8BBB0895AC
:1000B000B09902C08FEF089580E0089528E088E1AC
:1000C00090E00FB6F894A89581BD0FBE21BD85B70D
:1000D000877E806185BFFFCFEF92FF920F931F93C2
:1000E000DF93CF930F92CDB7DEB7AADF789485B7B1
:1000F000877E806185BF85B7806285BF889585B71B
:100100008F7D85BF92E080E80FB6F89486BD96BDDE
:100110000FBECE9B03C0FF24F39402C084E6F82EEA
:100120008BB78F7D8BBFC29A8FE493EC0197F1F769
:1001300000C00000BDDF882309F4C0DF80E090E04C
:1001400086D180958093600081E090E080D1809599
:10015000809361008091600095DF1091600090E0D5
:1001600000E0EE24E39429C0ABE7B2E91197F1F780
:1001700000C000009F5F063050F49B30E0F00F5F3E
:100180001F5F133008F010E0812F7CDF13C0943024
:1001900090F00F5F1F5F133008F010E0812F72DFC7
:1001A00081E090E054D18F3F19F01092610002C0BD
:1001B000E092610090E010936000998379DF99816B
:1001C000882391F686B1806C86B9DA9A89B7816006
:1001D00089BF809161008823E1F084E053DFE7EA82
:1001E000F1E63197F1F700C00000809160004ADF2E
:1001F00087EA91E60197F1F700C0000084E042DF52
:10020000A7EAB1E61197F1F700C000008091600005
:1002100039DFB299FECF8BB3877C8BBB80E09091A6
:100220006100992371F190916000923061F490E047
:1002300005C0BAE1BA95F1F700009F5F2091620016
:100240009217B8F36CC090916000913011F090E07B
:1002500013C090E005C0E4ECF0E03197F1F79F5F48
:10026000209162009217B8F35AC0A8EAB7E011973C
:10027000F1F700C000009F5F209162009217A8F381
:100280004EC0909160009230B9F490E005C0BAE1A0
:10029000BA95F1F700009F5F209162009217B8F3C2
:1002A00090E005C0E2E0EA95F1F700C09F5F209181
:1002B00063009217B8F333C090916000913011F051
:1002C00090E01EC090E005C0A4ECB0E01197F1F7FB
:1002D0009F5F209162009217B8F390E005C0BAE1E9
:1002E000BA95F1F700009F5F209163009217B8F371
:1002F00016C0E8EAF7E03197F1F700C000009F5F11
:10030000209162009217A8F390E005C0A4ECB0E041
:100310001197F1F79F5F209163009217B8F38F5FF9
:100320008F1508F47CCFC19A8BB388638BBB80E0B8
:1003300090916100992369F190916000923061F48D
:1003400090E005C0BAE1BA95F1F700009F5F2091F7
:1003500063009217B8F31DC090916000913011F0C6
:1003600090E013C090E005C0E4ECF0E03197F1F7C5
:100370009F5F209163009217B8F30BC0A8EAB7E023
:100380001197F1F700C000009F5F20916300921762
:10039000A8F38F5F8F1560F280916100882349F484
:1003A0008FED92E2A2E081509040A040E1F700C0C2
:1003B0000000C1988091600065DE8FE59AEEA0E0B4
:1003C00081509040A040E1F700C0000022CF189576
:1003D0001F920F920FB60F9211242F933F934F93BA
:1003E0005F936F937F938F939F93AF93BF93EF939D
:1003F000FF9387B1882331F485B18093630081E056
:1004000087B904C085B18093620017B851DE882394
:1004100069F060916000609580E090E020D060918C
:100420006100609581E090E01AD048DEFF91EF9185
:10043000BF91AF919F918F917F916F915F914F91FC
:100440003F912F910F900FBE0F901F901895E1993B
:10045000FECF1FBA8EBBE09A99278DB30895262F41
:10046000E199FECF1CBA1FBA8EBB2DBB0FB6F89414
:0E047000E29AE19A0FBE01960895F894FFCF2C
:00000001FF
